:020000040000FA
:02000000A02836
:08000800A000030EA100831209
:0C0010008101210E8300A00E200E0900CB
:10014000203084008001840A80300402031CA2282D
:100150006030AC00AD0083161E3085053330860557
:1001600083128501860107309F00C8308316810005
:100170008312313090007E30920026308316980032
:100180008312803098000C30831699008312BD10C2
:100190003D11BD15BD123D13BD17003083168C00F7
:1001A000831200308B0081018E018F010B118B10A7
:1001B0000B108C130C138C120C120C118C100C10D5
:1001C0008B173230A90062219E210510BC1A98219C
:1001D000BC1A0514A908031D0514031DA903A201D7
:1001E000A30186170330A7005621A70BF428061792
:1001F0000530A7005621A70BFA2806130310861E08
:100200000314A40D0530A7005621A70B0429861559
:100210000230A7005621A70B0A2986110230A70039
:100220005621A70B102986130530A7005621A70BCE
:1002300016290730A30006170330A7005621A70B85
:100240001E2906130310861E0314A40D0330A700F5
:100250005621A70B2829A30B1B292208403E840006
:100260000008A50024082506A60003194E29BC1B7A
:1002700041292608250503193F297E224929C02145
:10028000492926082505031D4729D52349293C234B
:1002900049292208403E8400250880000830A30038
:1002A000A20A203022020318E3281B2964000F1E33
:1002B00008008F018E01B108031D60297124080018
:1002C000B1030800BC01051DBC1785187229051A69
:1002D0008C29BC16BD103D11BD11851D3D1585191C
:1002E000BD150800851D8029051E7B29BC14BD1085
:1002F0003D11BD150800BC15BD103D11BD15080010
:10030000051E87293C15BD103D11BD1508003C1484
:10031000BD143D11BD110800851D9329BC15BD10EC
:100320003D15BD1108003C15BD103D15BD1108005F
:100330000030BC1B3130AF0060240800BD1CAA296E
:10034000BD1A08006730831699008312BD163D134D
:10035000BD1308003D1DB6293D1B0800193083164A
:1003600099008312BD123D17BD130800BD1B080084
:100370000C30831699008312BD123D13BD1708007F
:100380002208A800A80DA80DA80DF830A805260879
:10039000A70027180830A718073027190630A71913
:1003A0000530271A0430A71A0330271B0230A71B79
:1003B0000130A700A8073C1CE8292130AF006024C9
:1003C0002808AF0060242C08B0002030AF00602463
:1003D000BC1C162A5430AF0060242808AA008824C8
:1003E0002C30AF0060246730AF0060242C30AF00A9
:1003F00060243130AF0060240D30AF0060242C0841
:10040000B0005430AF0060242808AA0088242C30A3
:10041000AF0060246730AF0060242C30AF00602450
:100420003030AF0060240D30AF0060243C1D322A14
:100430007830AF0060249030AF0060242808AF000F
:100440006024C030AF0060242C08B0007830AF00CA
:1004500060249030AF0060242808AF006024803012
:10046000AF006024BC1D5D2A5230AF00602488308C
:10047000AA000310A80C03182A150310A80C0318CF
:10048000AA142808AF0060242A08AF0060242808B6
:10049000523A2A06AF0060242C08B0005230AF0058
:1004A0006024AA112808AF0060242A08AF00602445
:1004B0002808523A2A06AF006024013027020319A7
:1004C000A517023027020319251703302702031945
:1004D000A516043027020319251605302702031933
:1004E000A515063027020319251507302702031921
:1004F000A514083027020319251408002208A800B3
:10050000A80DA80DA80DF830A8052608A7002718E3
:100510000830A718073027190630A7190530271A01
:100520000430A71A0330271B0230A71B0130A70095
:10053000A8073C1CA62A2230AF0060242808AF0080
:1005400060242C08B0002030AF006024BC1CD42AEA
:100550005430AF0060242808AA0088242C30AF0053
:1005600060247230AF0060242C30AF006024313042
:10057000AF0060240D30AF0060242C08B000543070
:10058000AF0060242808AA0088242C30AF00602423
:100590007230AF0060242C30AF0060243030AF00E8
:1005A00060240D30AF0060243C1DF02A7830AF008D
:1005B00060249030AF0060242808AF0060244030F1
:1005C000AF0060242C08B0007830AF006024903079
:1005D000AF0060242808AF0060240030AF00602422
:1005E000BC1D1B2B5230AF0060248930AA000310C1
:1005F000A80C03182A150310A80C0318AA1428081D
:10060000AF0060242A08AF0060242808523A2A0666
:10061000AF0060242C08B0005230AF006024AA1153
:100620002808AF0060242A08AF0060242808523A46
:100630002A06AF006024013027020319A5130230F7
:10064000270203192513033027020319A5120430CA
:10065000270203192512053027020319A5110630B8
:10066000270203192511073027020319A5100830A6
:1006700027020319251008002208A800A80DA80DBC
:10068000FC30A80526180730A618063026190530B4
:10069000A6190430261A0330A61A0230261B013090
:1006A000A61B0030AB0003102B0CA700A807A80A5C
:1006B0002B183D142B1C3D103C1C6C2B3D1C213079
:1006C0003D182230AF0060242808AF0060242C08B9
:1006D000B0002030AF006024BC1C862B5430AF002B
:1006E00060242808AA0088242C30AF0060243D1C18
:1006F00067303D187230AF0060242C30AF006024AA
:100700003130AF0060240D30AF0060243C1D972BCA
:100710007830AF0060249030AF0060242808AF002C
:1007200060243D1CC0303D184030AF006024BC1D2B
:10073000B42B5230AF0060243D1C88303D18893006
:10074000AA000310A80C03182A150310A80C0318FC
:10075000AA142808AF0060242A08AF0060242808E3
:10076000523A2A06AF00602400302B020319A51369
:1007700001302B020319251302302B020319A51295
:1007800003302B020319251204302B020319A51183
:1007900005302B020319251106302B020319A51071
:1007A00007302B020319251008002208A800A80D05
:1007B000A80DFC30A80526180730A6180630261903
:1007C0000530A6190430261A0330A61A0230261B5B
:1007D0000130A61B0030AB0003102B0CA700A807AC
:1007E000A80A2B183D142B1C3D103C1CF72BBC1CDD
:1007F000112C5430AF0060242808AA0088242C3023
:10080000AF0060243D1C67303D187230AF0060249B
:100810002C30AF0060243030AF0060240D30AF00CA
:1008200060243C1D222C7830AF0060249030AF0053
:1008300060242808AF0060243D1C80303D18003043
:10084000AF006024BC1D3F2C5230AF0060243D1C23
:1008500080303D188130AA000310A80C03182A1517
:100860000310A80C0318AA142808AF0060242A0853
:10087000AF0060242808523A2A06AF0060240030F6
:100880002B020319A51701302B020319251702307B
:100890002B020319A51603302B0203192516043069
:1008A0002B020319A51505302B0203192515063057
:1008B0002B020319A51407302B0203192514080075
:1008C000A908031D080020302E02031808002C0878
:1008D00084002F088000AE0AAC0A6030AC1BAC006C
:1008E00008000C1E0800AE080319080005142D08A6
:1008F000840000089900AE03AD0A6030AD1BAD0066
:100900002D083002031D08004630B100B001080078
:100910000A302A02031CA22C64302A02031C9F2CDA
:10092000C8302A02031C9A2CC830AA023230AF0009
:1009300060249F2C6430AA023130AF006024A624CA
:10094000AF006024AB24AF0060240800AA13053078
:100950008A002A088200AA1705308A002A08820025
:100A000030343034303430343034303430343034C6
:100A100030343034313431343134313431343134B0
:100A2000313431343134313432343234323432349A
:100A30003234323432343234323432343334333484
:100A4000333433343334333433343334333433346E
:100A50003434343434343434343434343434343456
:100A60003434343435343534353435343534353440
:100A7000353435343534353436343634363436342A
:100A80003634363436343634363436343734373414
:100A900037343734373437343734373437343734FE
:100AA00038343834383438343834383438343834E6
:100AB00038343834393439343934393439343934D0
:100AC00039343934393439343034303430343034E2
:100AD00030343034303430343034303431343134F4
:100AE00031343134313431343134313431343134DE
:100AF00032343234323432343234323432343234C6
:100B000030343134323433343434353436343734A9
:100B10003834393430343134323433343434353495
:100B20003634373438343934303431343234333481
:100B3000343435343634373438343934303431346D
:100B40003234333434343534363437343834393459
:100B50003034313432343334343435343634373459
:100B60003834393430343134323433343434353445
:100B70003634373438343934303431343234333431
:100B8000343435343634373438343934303431341D
:100B90003234333434343534363437343834393409
:100BA0003034313432343334343435343634373409
:100BB00038343934303431343234333434343534F5
:100BC00036343734383439343034313432343334E1
:100BD00034343534363437343834393430343134CD
:100BE00032343334343435343634373438343934B9
:100BF00030343134323433343434353436343734B9
:084000000E00010000000200A7
:02400E00543D1F
:00000001FF
